:1000000000308A0083280000831A0A288E00030E1D
:100010008F000F2883128E00030E8F008F140A08A2
:1000200093008A0183138E0E040890000C0891003F
:100030000D08920083128B1E1F280B1943281008ED
:10004000840011088C0012088D0013088A000F0E1E
:10005000830083120E0E8F18831609001F30840050
:1000600000080319422801308D008C018C0B3628C2
:100070008D0B35284A308C008C0B3C28000000008A
:10008000800B3328003418148316051183120515CC
:1000900001309F002E2016089E009E08031952284A
:1000A0009E034D2814089E009E0803195E28063002
:1000B0008C008C0B592800009E03542883160511D0
:1000C00083120511831606108312061401309F0057
:1000D0002E2017089E009E08031970289E036B2887
:1000E00015089E009E0803197C2806308C008C0B96
:1000F000772800009E0372288316061083120610CC
:100100000B118A111F2884011F30830510309400C1
:10011000950002309600970005308C008C1D9828C1
:1001200007308101813084000008C0390F38800019
:100130006400813084000008C0390C0480008B16F4
:100140008B1718100F30990099080319B82814302C
:100150008C008C0BA9280000181CAF28A12883163E
:10016000851583128519B6280F3099009903A428A4
:10017000831685158312851DC128181CC028A12847
:10018000B828181CC428A128DD308C008C0BC62888
:10019000000000000830990099080319E9280310AD
:1001A0009B0D831685158312851DD7281B14181CDB
:1001B000DA28A1288316861083128614AB308C00AF
:1001C0008C0BE0280000831686108312861099039A
:1001D000CC289C01043099009908031909290310BF
:1001E0009C0D831685158312851DF7281C14181C79
:1001F000FA28A1288316861083128614AB308C004F
:100200008C0B002900008316861083128610990338
:10021000EC289B0E1B080F399D009B0E1B080F3905
:100220009D079D0A0F309D051C081D020319192901
:10023000A1281B0E9A009A0C07309A051F309B05C7
:1002400001301A02FE3E03182D29023E2F291B08F9
:1002500094002D291B0895002D29A12863000A145C
:0A0260008A100A11820727292A29B3
:02400E00F13F80
:00000001FF
